:0200000480007A
:100000006F008004732F2034930F80006308FF0378
:10001000930F90006304FF03930FB0006300FF038E
:10002000130F000063040F0067000F00732F2034CC
:1000300063540F006F00400093E19153171F0000BD
:1000400023223FFC6FF09FFF93000000130100008C
:10005000930100001302000093020000130300004C
:100060009303000013040000930400001305000034
:10007000930500001306000093060000130700001C
:100080009307000013080000930800001309000004
:1000900093090000130A0000930A0000130B0000EC
:1000A000930B0000130C0000930C0000130D0000D4
:1000B000930D0000130E0000930E0000130F0000BC
:1000C000930F0000732540F16310050097020000B4
:1000D000938202017390523073500018970200000F
:1000E00093824202739052309B021000939252030B
:1000F0009382F2FF7390023B9302F0017390023AF5
:100100007350403097020000938242017390523046
:10011000735020307350303093010000970200007C
:10012000938282EE73905230130510001315F5017F
:10013000635C05000F00F00F930110009308D005D9
:10014000130500007300000093020000638A0200A0
:1001500073905210B7B200009B82921073902230BD
:100160007350003037250000732005307350300085
:10017000970200009382420173901234732540F17C
:1001800073002030172400001304C4E70731040073
:1001900027382400033504019B0310009393730256
:1001A0009383F317939373019301200063187508E9
:1001B0000731040027282400033504019B031000A5
:1001C000939373029383F317939373019301300016
:1001D000631675060721040027282400033504014F
:1001E0009B031000939373029383F317939373010C
:1001F00093014000631475040731840027382400FC
:10020000033504019B0310F8939313029383131097
:1002100093936301930150006312750207218400D8
:1002200027382400033504019B0310D09393630106
:100230009301600063147500631030020F00F00F2B
:10024000638001009391110093E111009308D005A0
:1002500013850100730000000F00F00F93011000E0
:100260009308D0051305000073000000731000C050
:0C02700000000000000000000000000082
:1010000000000000000000000000000000000000E0
:1010100000000000000000000000000000000000D0
:1010200000000000000000000000000000000000C0
:1010300000000000000000000000000000000000B0
:081040000000000000000000A8
:10200000000080BF0000004000004040000080C091
:10201000EFBEADDEBEBAFECAEA1DADAB0DD03713C2
:040000058000000077
:00000001FF
